:100000000C9483020C94C7020C94C7020C94C70290
:100010000C94C7020C94C7020C94C7020C94C7023C
:100020000C94C7020C94C7020C94960D0C94680EA5
:100030000C94C7020C94C7020C94C7020C94C7021C
:100040000C94C7020C9472220C94C7020C94C70241
:100050000C94C7020C94051C0C94C7020C94C702A4
:100060000C94C7020C94C7020C94C7020C94C702EC
:100070000C94C7020C94C7020C94C7020C94C702DC
:100080000C94C7020C94C7020C94C7020C94C702CC
:100090000C94C7020C94C7020C94C7020C94C702BC
:1000A0000C94C7020C94C7020C94C702D50EF70E2D
:1000B000E50FF70EE50F3C0F5F0FE50FB40FC70F0D
:1000C00096129612C512C512FB121B134C144C1437
:1000D00026134C14D613D6133D144C144C1446144A
:1000E000E313E313E313E313E313E313E313E31360
:1000F000E313E313E313E313E313E313E313E31350
:10010000F5130214091410141A1401E40135023510
:1001100002E40001E00104020402E00000C801C89A
:1001200035002B00E300E100002000001E00140059
:1001300004001D002F024D001F001A0016001B00B6
:1001400026022900200008000700060031022A00CC
:10015000210015000900190033024A00220017008F
:100160000A0005000000E2083E002F0000000154D4
:100170000000E200100F3000000002540000E60012
:1001800023001C000B0011000000AE00240018002A
:100190000D0010002D004B0025000C000E00360055
:1001A0002E002C00260012000F0037002702280026
:1001B000270013003300380030024E00A800310041
:1001C0003400E500012000000100010001000100F1
:1001D000010000003A001E0220022202010001007C
:1001E0003B001F0221022302010001003C002F02FC
:1001F00026022F00010001003D00300227023000DE
:10020000010001003E00310235003502000001000E
:1002100001000100000001000000010001000100D8
:1002200000000100000001003F000100500001003B
:100230000000010040000100510001000100010028
:1002400041000100520001000100010042000100D4
:100250004F00010001000100430001000100010006
:100260000100010044004500010001000100000000
:100270000100010001000100A900000001000100CF
:1002800001000100AA0001000100010001000100BD
:10029000AC0001000100010001000100AB00010001
:1002A0000100010001000100010001000100010046
:1002B0000100010000000100010001000000010038
:1002C0000000010001000100000001000000010029
:1002D00001000100F2000100000001000100010026
:1002E000F1000100F400010001000100F000010034
:1002F000F500B60001000100F3000100010001005B
:1003000001000100010001000100010001000100E5
:1003100001000100010000001603450072006700A3
:100320006F0044006F007800200045005A00000074
:1003300016034500720067006F0044006F007800EC
:10034000200045005A0000000403090409026D0062
:10035000040100A0FA0904000001030101000921C1
:1003600011010001223F000705810308000A09046A
:1003700001000103010200092111010001224D00C9
:100380000705820308000A090402000103000000B7
:100390000921110100012236000705830308000A24
:1003A00009040300010300000009211101000122DA
:1003B000390007058403100001120110010000003C
:1003C00008EDFE071301000102000105010906A165
:1003D00001050719E029E715002501950875018138
:1003E0000205081901290595057501910295017508
:1003F00003910105071900297715002501957875E6
:10040000018102C005010980A101850216010026B3
:10041000B7001A01002AB700751095018100C005C8
:100420000C0901A1018503160100269C021A010096
:100430002A9C02751095018100C005010902A101E5
:100440000901A100050919012905150025019505D6
:10045000750181029501750381010501093009319A
:100460001581257F95027508810609381581257F3C
:10047000950175088106050C0A38021581257F95BE
:100480000175088106C0C005010906A1010507190B
:10049000E029E71500250195087501810295017590
:1004A0000881010508190129059505750191029535
:1004B00001750391010507190029FF150025FF9516
:1004C0000675088100C00000000000000000000068
:1004D00000010204060A0F17202C3A4A5D71879D1D
:1004E000B3C7DAE9F5FCFFFCF5E9DAC7B39D87711C
:1004F0005D4A3A2C20170F0A060402010000000092
:1005000000000000000011241FBECFEFDAE0DEBFC4
:10051000CDBF04B603FE24C08091FB019091FC0185
:10052000A091FD01B091FE018730904BA740B04BE8
:10053000B9F41092FB011092FC011092FD0110928F
:10054000FE0114BE84B7877F84BF88E10FB6F8949C
:1005500080936000109260000FBEE0E0FFE3099519
:1005600011E0A0E0B1E0E2E7F8E402C005900D92EE
:10057000A433B107D9F711E0A4E3B1E001C01D92A3
:10058000AB3FB107E1F70E94DA0A0C9437240C94D0
:1005900000001092B9008AE08093B800089594EAB0
:1005A0009093BC009091BC0097FFFCCF9091B90054
:1005B000987F983021F0903111F081E00895809378
:1005C000BB0084E88093BC008091BC0087FFFCCF17
:1005D0008091B900887F883111F0803471F780E014
:1005E000089584E98093BC008091BC0084FDFCCF19
:1005F00008958093BB0084E88093BC008091BC0088
:1006000087FFFCCF9091B900987F81E0983209F480
:1006100080E0089584E88093BC008091BC0087FF4F
:10062000FCCF8091BB00089580910101811115C01C
:1006300080E40E94CF028093010181110CC082E10D
:100640000E94F90280930101811105C08FEF0E9481
:10065000F902809301010E94F10284B1807F84B984
:1006600085B1807F85B98AB1837F8AB98BB1837F59
:100670008BB93E98469808950E94CF04809301015B
:100680000E94140380B38C7080BB81B3836F81BBE5
:10069000A5E3B1E0E3E4F1E08EE08E0F11921D924C
:1006A0008E13FCCF0C94B904BF92CF92DF92EF92DD
:1006B000FF920F931F93CF93DF93809101018823C3
:1006C00079F0809134018F5F80933401811108C0EB
:1006D0000E94CF0480930101811102C00E94610435
:1006E00005E311E0C0E0D0E0DD24D39482E0C82E21
:1006F000EE24E394F12CC730D10500F5809101017F
:10070000811164C080E40E94CF02809301018111B5
:1007100012C082E10E94F9028093010181110BC095
:10072000C7010C2E01C0880F0A94EAF780950E9439
:10073000F902809301010E94F10248C0CA30A1F081
:1007400028F4C83059F0C93061F005C0CC3089F0C8
:1007500070F0CD3089F0209A289810C0219A2998FD
:100760000DC0229A2A980AC0239A2B9807C0529A41
:1007700001C0539A5B9802C03E9A469890EA9A95B7
:10078000F1F79FB1799902C082E001C080E09170D9
:100790009D25982B7C9902C084E001C080E0892BC4
:1007A0007D9902C038E001C030E0832B7E9902C001
:1007B00020E101C020E0822B9FB19095991F9927DD
:1007C000991F9295990F907E892B0FC080910101FE
:1007D000811149C080E40E94CF02809301018823E7
:1007E00079F1B12C0E94F1028B2DF80190819817BC
:1007F00019F08083C09200010E94140321960F5FBC
:100800001F4FCE30D10509F076CF809100018823AB
:1008100061F1815080930001882339F08FE99FE0D6
:100820000197F1F700C0000020C0A3E4B1E0E5E3C8
:10083000F1E0CF01825F91919D938E13FCCF15C0A3
:1008400083E10E94F902809301018111CACF81E402
:100850000E94CF02809301018111C3CF0E940A033D
:10086000B82EB094BFCF80E0C0CF0E945F0481E07B
:10087000DF91CF911F910F91FF90EF90DF90CF907C
:10088000BF900895E82FF0E0ED5BFE4F8081089562
:1008900008950F931F93CF93DF93C3E4D1E010E04B
:1008A0000C2F025F899190E00E942B1B180F0C13F4
:1008B000F9CF812FDF91CF911F910F9108950C9463
:1008C0005A0556985E9825982D9826982E98279820
:1008D0002F988FEF90E090938900809388009093F9
:1008E0008B0080938A0090938D0080938C00259AD2
:1008F0002D9A2FEF80E792E0215080409040E1F761
:1009000000C00000269A2E9A2FEF80E792E0215037
:1009100080409040E1F700C00000279A2F9A2FEF07
:1009200080E792E0215080409040E1F700C0000055
:1009300025982D982FEF80E792E02150804090403D
:10094000E1F700C0000026982E982FEF80E792E094
:10095000215080409040E1F700C0000027982F9878
:1009600056985E9825982D9826982E9827982F9817
:10097000089589EA8093800089E08093810024981B
:100980002C983F988AB18F748AB96E98479A8BB128
:10099000806B8BB9769A0E9461040C94590580E2B1
:1009A000809301018091510181110EC00E94C90202
:1009B00081E0809351012FEF83ED90E3215080403F
:1009C0009040E1F700C0000080E40E94CF028093D5
:1009D000010181112EC00E94F90280930101811151
:1009E00028C00E94F90280930101811122C08FE387
:1009F0000E94F9028093010181111BC00E94F10243
:100A000080E40E94CF0280930101811112C08CE02A
:100A10000E94F9028093010181110BC00E94F9022A
:100A200080930101811105C08FE30E94F902809338
:100A300001010E94F102809101010895CF93DF939B
:100A4000EC01662319F06130C9F015C09A818D81DF
:100A5000992349F0982F907F21F080FF22C08F705A
:100A60008D8380EE17C0807F19F480EE0E94021201
:100A70008D818F708D8380E090E018C09A818D8188
:100A8000992359F0982F907F21F080FF0DC08F702F
:100A90008D8384EE0E943A11EECF807F49F784EE79
:100AA000E5CF83E191E002C08AE091E0DF91CF9150
:100AB000089508956091BD017091BE018091BF01BC
:100AC0009091C0010E94371B56985E9825982D98EA
:100AD00026982E9827982F98813019F0823021F08F
:100AE0000895259A2D9A0895269A2E9A089581E0C0
:100AF000089581E008950C94790508950F931F934C
:100B0000CF93DF938C01FC01C081D181CE010E9483
:100B1000B019BE010E942706EC01B8010E947B05B6
:100B2000882309F48DC0F8018281882309F44AC022
:100B300080915D0181111FC0C431F0E5DF0709F02C
:100B400051C00E947D0581E080935D010E94CF1B12
:100B500090935C0180935B011092540110925601B6
:100B600010925501109258011092570110925A019B
:100B70001092590165C080915B0190915C010E94C7
:100B8000DB1B883C910570F480915401E82FF0E064
:100B9000EE0FFF1FEB5AFE4FD183C0838F5F809310
:100BA00054014EC0C43880E5D80721F0C538D0457F
:100BB00001F13AC0F8018281882341F0109252017C
:100BC00082E01EC0C438E0E5DE0759F5809152018D
:100BD000811106C086E20E943A1186E20E9402124A
:100BE00082E01CC0C438F0E5DF0741F3C538D045CA
:100BF000D9F4F8018281882331F01092530180E208
:100C00000E9451121DC080915301811106C087E2DC
:100C10000E943A1187E20E94021280E20E9458125A
:100C20000FC0C538D04529F381E0809352018093ED
:100C30005301C801DF91CF911F910F910C9477055B
:100C400080E0DF91CF911F910F910895089596E074
:100C5000799FF001112494E5899FE00DF11D112485
:100C6000E60FF11DEE0FFF1FE05EFE4F85919491A0
:100C70000895880F991FFC01E456F04085919491E6
:100C80000895880F991FFC01E45EFE4F85919491B1
:100C900008950F931F93CF93DF93EC01811520E309
:100CA000920750F5C11580E2D80708F0C3C0CB3BCE
:100CB000D10590F4C83AD10508F06AC0C53AD1050B
:100CC00008F05BC0C430D10508F0D0C1219709F00D
:100CD000CAC101E010E00AC2CF3FD10511F008F00F
:100CE000C5C1C03FD10508F0A2C0CE01805E910908
:100CF000089708F4BBC1B7C1C13090E5D90709F422
:100D0000A2C020F5C0318FE4D80770F4C11590E47B
:100D1000D90708F094C0C11521E3D20708F0A3C198
:100D2000DD278E01106CE2C1C115D04509F09BC1D1
:100D30000E94B7148FEF94E32CE081509040204044
:100D4000E1F700C000000E942A1CD0C1C11597E540
:100D5000D90758F4C03121E5D20708F01CC1C431CD
:100D600080E5D80708F475C07EC1CE019057811583
:100D7000904108F078C1DF7073C1C53AD10509F41C
:100D800077C1C63AD10509F076C102E810E4AEC1D8
:100D9000C83AD10509F472C1C93AD10509F471C143
:100DA000CA3AD10509F470C1CB3AD10509F46FC133
:100DB000CC3AD10509F46EC1CD3AD10509F46DC123
:100DC000C03BD10509F46CC1CE3AD10509F46BC121
:100DD000CF3AD10509F46AC1C13BD10509F469C113
:100DE000C23BD10509F468C1C33BD10509F467C111
:100DF000C43BD10509F466C1C53BD10509F465C101
:100E0000C63BD10509F464C1C73BD10509F463C1F0
:100E1000C83BD10509F462C1C93BD10509F461C1E0
:100E2000CA3BD10509F460C100E014E45FC18E0142
:100E300010655CC1CE019F700E94410658C1DF70F1
:100E40008E01106A53C18091DA0181608093DA01CA
:100E50004DC10E94CF1D811102C00E94B51D0E948C
:100E6000EC1D90E09093FB018093FA01C23080E585
:100E7000D80721F48091FA01816086C0C43090E5E2
:100E8000D90721F48091FA0182607EC0C63020E546
:100E9000D20721F48091FA01846076C0C83080E5E1
:100EA000D80719F48091FA0127C0CA3090E5D90714
:100EB00021F48091FA01806167C0CC3020E5D2072F
:100EC00021F48091FA0180625FC0CE3080E5D807BE
:100ED00021F48091FA01806457C0C03190E5D907B0
:100EE00021F48091FA0180684FC0C23120E5D20719
:100EF00029F48091FA018460886046C0C33080E59F
:100F0000D80721F48091FA018E7F3EC0C53090E56C
:100F1000D90721F48091FA018D7F36C0C73020E5D2
:100F2000D20721F48091FA018B7F2EC0C93080E571
:100F3000D80719F48091FA0126C0CB3090E5D90783
:100F400021F48091FA018F7E1FC0CD3020E5D207B9
:100F500021F48091FA018F7D17C0CF3080E5D8074A
:100F600021F48091FA018F7B0FC0C13190E5D90740
:100F700021F48091FA018F7707C0C331D04531F455
:100F80008091FA018B7F877F8093FA018091FA012B
:100F90000E94F01DABC08D2F99278F70992781304B
:100FA0009105D9F49E012370332702C0880F991F41
:100FB0002A95E2F79C688E0144E0000F111F4A95C4
:100FC000E1F700271370802B912B53E0CC0FDD1F2E
:100FD0005A95E1F7C076DD272FC08230910531F4B4
:100FE000DC2FCC278E01016F106A80C08330910501
:100FF00069F4CE018370992701E010E002C0000F70
:10100000111F8A95E2F7C8019C680FC084309105D2
:10101000B9F4CE018370992701E010E002C0000FFF
:10102000111F8A95E2F7C8019A6823E0CC0FDD1FF3
:101030002A95E1F7C07ED7708C010C2B1D2B56C072
:101040008530910531F4DC2FCC278E01046F106AB6
:101050004DC0069709F04AC0CF71DD27DC2FCC27A1
:101060008E01106243C000E010E040C08E013EC01F
:1010700001E810E43BC003E810E438C002EE14E4D9
:1010800035C009EE14E432C00AEE14E42FC005EBBB
:1010900014E42CC006EB14E429C007EB14E426C0CA
:1010A0000CEC14E423C00DEC14E420C003E815E4B8
:1010B0001DC00AE815E41AC002E915E417C004E9E6
:1010C00015E414C001E216E411C003E216E40EC0F8
:1010D00004E216E40BC005E216E408C006E216E4DA
:1010E00005C007E216E402C00AE216E4C801DF9177
:1010F000CF911F910F91089596E0799FF0011124EF
:1011000094E5899FE00DF11D1124E60FF11DEE0F0E
:10111000FF1FE05EFE4F85919491803E9105E0F4C3
:10112000803C910558F58133910509F46FC048F46E
:101130008932910509F463C08A32910509F46DC0C2
:1011400072C089339105E9F082389105D1F0853379
:10115000910509F44DC067C0833E910581F138F4D3
:10116000803E9105B9F0823E9105D9F05CC0863E83
:10117000910561F1873E9105A1F155C00E943906A4
:1011800008952091FA0120FD02C021FF4CC080EE9D
:1011900090E049C08091FA0180FFF9CF89E390E0A7
:1011A00042C08091FA0182FF0EC08091FA0184FF53
:1011B00003C080E090E037C083EE90E034C08091BF
:1011C000FA0182FFF2CF82EE90E02DC08091FA0109
:1011D00083FF0BC08091FA0184FDEBCF87EE90E096
:1011E00022C08091FA0183FFF5CF86EE90E01BC00C
:1011F0008091FA0185FF07C089E290E014C08091D8
:10120000FA0185FFF9CF85E390E00DC08091FA01E6
:1012100086FF07C08AE290E006C08091FA0186FF4F
:10122000F9CF81E390E00E944906089508950C9457
:10123000160980916E010895CF93DF9300D01F921D
:10124000CDB7DEB79C018091F101843019F593E0B0
:1012500099833B832A839093E9008FEF9091E80074
:10126000815095FD06C095ED9A95F1F7000081112A
:10127000F5CF8091E80085FF0DC040E050E063E0CD
:1012800070E0CE0101960E94860B8091E8008E7777
:101290008093E8000F900F900F90DF91CF91089509
:1012A000CF93DF9300D01F92CDB7DEB72091F1012D
:1012B000243021F522E029839B838A8383E0809375
:1012C000E9008FEF9091E800815095FD06C095ED03
:1012D0009A95F1F700008111F5CF8091E80085FF24
:1012E0000DC040E050E063E070E0CE0101960E9446
:1012F000860B8091E8008E778093E8000F900F9026
:101300000F90DF91CF9108952091F1012430F1F4F5
:1013100022E02093E9002FEF3091E800215035FDC5
:1013200006C035ED3A95F1F700002111F5CF209177
:10133000E80025FF0BC040E050E065E070E00E944F
:10134000860B8091E8008E778093E8000895CF9314
:10135000DF93EC019091F101943009F046C0809147
:101360000C018823D9F080910D018823B9F0909366
:10137000E9008FEF9091E800815095FD06C095E15E
:101380009A95F1F700008111F5CF8091E80085FF73
:101390002CC040E050E060E170E017C081E0809335
:1013A000E9008FEF9091E800815095FD06C095ED22
:1013B0009A95F1F700008111F5CF8091E80085FF43
:1013C00014C040E050E068E070E0CE010E94860B5F
:1013D0008091E8008E778093E80080E1FE01AEE521
:1013E000B1E001900D928A95E1F7DF91CF910895D8
:1013F0008091F001811109C00E941B0D0E94780D9F
:101400008091E20084608093E20008951092F001E0
:10141000089508950C945F220E94C01B0E946522CB
:101420000E941E100C94170942E061EC81E00E94BA
:10143000950C42E061EC82E00E94950C42E061EC88
:1014400083E00E94950C42E161EC84E00C94950CE1
:101450008091F301833009F455C030F4813071F08C
:10146000823009F48EC008958A3009F47AC08B3036
:1014700009F460C0893009F09CC020C08091F2015D
:10148000813A09F096C08091E800877F8093E80058
:101490008091F6019091F701892B21F460E18EE5AE
:1014A00091E003C060E080E090E070E00E94D10B2A
:1014B0008091E8008B778093E80008958091F20195
:1014C000813209F076C08091F6019091F701009782
:1014D00019F0039709F06DC08091E800877F809331
:1014E000E8008091E80082FD05C08091F101811142
:1014F000F8CF5FC08091F10080936E018091E80089
:101500008B7753C08091F201813A09F052C08091EB
:10151000F6019091F701892B09F04BC08091E8000A
:10152000877F8093E8008091E80080FFFCCF809166
:101530000C0136C08091F2018132D9F58091F6011B
:101540009091F701892BA9F58091E800877F80931E
:10155000E8000E94CA0C8091F40180930C010C9465
:10156000B7148091F201813221F58091E800877FE4
:101570008093E8000E94CA0C8091F50180936F016E
:1015800008958091F201813AA1F48091E800877F6B
:101590008093E8008091E80080FFFCCF80916F018C
:1015A0008093F1008091E8008E778093E8000C949E
:1015B000CA0C089584B7877F84BF88E10FB6F8947A
:1015C00080936000109260000FBE90E080E80FB63C
:1015D000F89480936100909361000FBE0E946D109B
:1015E0000E941B0D0E94780D8091E2008460809320
:1015F000E20078940E94FE0F0E946F1082E091E05A
:101600000E9419100E944D228091F101853069F4E9
:101610000E94871B8091EF018823B1F30E94B21BC7
:10162000882391F30E94700BEFCF0E947510ECCFCE
:10163000292F332723303105C9F064F421303105D7
:1016400081F02230310509F043C08DE690E02CE4B2
:1016500033E042C021323105F1F02232310541F14F
:1016600037C082E190E029EB33E036C09927813022
:10167000910541F08230910541F0892B49F5E8E46C
:10168000F3E005C0E0E3F3E002C0E8E1F3E08491B9
:1016900090E09F0121C06430D8F4E62FF0E0EE0F17
:1016A000FF1FEE5DFE4F2081318189E090E014C084
:1016B000643070F470E0FB01EE0FFF1FE65EFE4F3A
:1016C00020813181FB01EA5EFE4F808190E004C001
:1016D00080E090E020E030E0FA013183208308953B
:1016E00080E189BD82E189BD09B400FEFDCF809112
:1016F000D8008F7D8093D8008091E0008260809335
:10170000E0008091E00081FDFCCF0895CF92DF9250
:10171000EF92FF920F931F93CF93DF93EC018B0116
:101720006A010E94E90C811133C0C114D10439F05F
:10173000F60180819181081B190BC80FD91FE12C7C
:10174000F12C0115110519F18091E80085FD16C0F5
:101750008091E8008E778093E800C114D10449F0AD
:10176000F60180819181E80EF91EF182E08285E028
:101770000FC00E94E90C882321F30AC0899180934D
:10178000F10001501109FFEFEF1AFF0ADACF80E0F4
:10179000DF91CF911F910F91FF90EF90DF90CF904D
:1017A00008952091F8013091F9012617370748F084
:1017B0006115710539F42091E8002E772093E80037
:1017C00001C0B90140E061157105A9F12091F10155
:1017D000222309F443C0253009F442C02091E800D7
:1017E00023FD40C02091E80022FD32C02091E80096
:1017F00020FFE9CF4091F3002091F20030E0342B3C
:10180000FC01CF016115710559F02830310540F414
:1018100081918093F100615071092F5F3F4FF1CFAB
:1018200041E02830310509F040E02091E8002E77B2
:101830002093E800C8CF4111C9CF0AC08091F101BF
:10184000882361F0853061F08091E80083FD0AC053
:101850008091E80082FFF2CF80E0089582E0089551
:1018600083E0089581E008952091F8013091F90115
:101870002617370748F06115710539F42091E80003
:101880002E772093E80001C0B901FC0120E061152A
:10189000710591F18091F101882309F440C08530F0
:1018A00009F43FC08091E80083FD3DC08091E800CD
:1018B00082FD2FC08091E80080FFE9CF2091F300E6
:1018C0008091F20090E0922B6115710559F08830FB
:1018D000910540F424912093F100319661507109F3
:1018E0000196F2CF21E0089709F020E08091E8000E
:1018F0008E778093E800CBCF2111CCCF0AC08091A6
:10190000F101882361F0853061F08091E80083FD6A
:101910000AC08091E80082FFF2CF80E0089582E063
:10192000089583E0089581E00895982F973058F541
:101930009093E900981739F07091EC002091ED0038
:101940005091F00003C0242F762F50E021FF19C0E2
:101950003091EB003E7F3093EB003091ED003D7F06
:101960003093ED003091EB0031603093EB007093D9
:10197000EC002093ED005093F0002091EE0027FF43
:1019800007C09F5FD3CF8F708093E90081E00895F7
:1019900080E008958091F20187FF11C08091E800F6
:1019A00082FD05C08091F1018111F8CF11C08091B5
:1019B000E8008B770BC08091F101882349F080917A
:1019C000E80080FFF8CF8091E8008E778093E800F0
:1019D00008952091E4003091E50095E64091EC00F7
:1019E000842F817040FF22C08091E80080FD1CC0E0
:1019F0008091F101882391F0853091F08091EB0086
:101A000085FD10C04091E4005091E5004217530756
:101A100029F39A01915011F784E0089582E0089526
:101A200083E0089581E0089580E008954091E80002
:101A300042FFDECF08950E94890D0E94910DE0EED5
:101A4000F0E0808181608083E8EDF0E080818F7735
:101A5000808319BCA7EDB0E08C918E7F8C93808140
:101A60008F7E80831092F00108950F931F93CF9380
:101A7000DF930E94890D0E94910DC8EDD0E088810E
:101A80008F77888388818068888388818F7D888329
:101A900019BC1092F1011092ED011092EF01109219
:101AA000EE0100EE10E0F80180818B7F8083888159
:101AB0008160888342E060E080E00E94950CE1EE66
:101AC000F0E080818E7F8083E2EEF0E080818160B3
:101AD0008083808188608083F80180818E7F80830D
:101AE000888180618883DF91CF911F910F91089544
:101AF000E8EDF0E080818F7E8083E7EDF0E080818B
:101B00008160808384E082BF81E08093F0010C9447
:101B1000350DE8EDF0E080818E7F80831092E20049
:101B200008951092DA001092E10008951F920F922A
:101B30000FB60F9211242F933F934F935F936F93A0
:101B40007F938F939F93AF93BF93EF93FF93809176
:101B5000E10082FF0BC08091E20082FF07C080910C
:101B6000E1008B7F8093E1000E94FD0F8091DA00FD
:101B700080FF1FC08091D80080FF1BC08091DA00D9
:101B80008E7F8093DA008091D90080FF0DC080E1C4
:101B900089BD82E189BD09B400FEFDCF81E080935B
:101BA000F1010E94F80905C019BC1092F1010E94D0
:101BB000060A8091E10080FF19C08091E20080FF59
:101BC00015C08091E2008E7F8093E2008091E20058
:101BD00080618093E2008091D80080628093D80079
:101BE00019BC85E08093F1010E940A0A8091E1000E
:101BF00084FF30C08091E20084FF2CC080E189BD69
:101C000082E189BD09B400FEFDCF8091D8008F7DAF
:101C10008093D8008091E1008F7E8093E1008091D5
:101C2000E2008F7E8093E2008091E20081608093E9
:101C3000E2008091ED01882311F084E007C08091DB
:101C4000E30087FD02C081E001C083E08093F101E1
:101C50000E940C0A8091E10083FF29C08091E2007C
:101C600083FF25C08091E100877F8093E10082E0BF
:101C70008093F1011092ED018091E1008E7F8093BD
:101C8000E1008091E2008E7F8093E2008091E2008B
:101C900080618093E20042E060E080E00E94950C69
:101CA0008091F00088608093F0000E94090AFF9103
:101CB000EF91BF91AF919F918F917F916F915F91C4
:101CC0004F913F912F910F900FBE0F901F9018953D
:101CD0001F920F920FB60F9211242F933F934F93A1
:101CE0005F936F937F938F939F93AF93BF93CF93A4
:101CF000DF93EF93FF93C091E900CF708091EC00E8
:101D0000D82FD17080FDD0E81092E9008091F000CA
:101D1000877F8093F00078940E94AC0E1092E900C7
:101D20008091F00088608093F000CD2BCF70C0933D
:101D3000E900FF91EF91DF91CF91BF91AF919F911A
:101D40008F917F916F915F914F913F912F910F9064
:101D50000FBE0F901F9018951F93CF93DF93CDB7B1
:101D6000DEB7AA970FB6F894DEBF0FBECDBFE2EF85
:101D7000F1E088E08E0F9091F10091938E13FBCFEC
:101D80000E94280A8091E80083FF1FC18091F20120
:101D90009091F301492F50E04A30510508F015C1E8
:101DA000FA01EA5AFF4F0C94E723803881F0823819
:101DB00009F00BC18091F6018F708093E90080914A
:101DC000EB0085FB882780F91092E90006C080911E
:101DD000EE019091EF01911182609091E800977F60
:101DE0009093E8008093F1001092F100C8C0282F72
:101DF0002D7F09F0EAC0882319F0823061F0E5C038
:101E00008091F401813009F0E0C0933009F080E066
:101E10008093EF012BC08091F401811127C0809144
:101E2000F6018F7009F4D1C08093E9002091EB0096
:101E300020FF1CC0933021F48091EB00806214C01D
:101E40009091EB0090619093EB0021E030E0A901CC
:101E500002C0440F551F8A95E2F74093EA001092A2
:101E6000EA008091EB0088608093EB001092E9001B
:101E70008091E800877F86C08111A7C01091F4018E
:101E80001F778091E3008078812B8093E30080911D
:101E9000E800877F8093E8000E94CA0C8091E800E8
:101EA00080FFFCCF8091E30080688093E3001111F4
:101EB00002C082E001C083E08093F10186C08058B7
:101EC000823008F082C08091F4019091F5018C3D40
:101ED00053E0950779F583E08A838AE289834FB7D7
:101EE000F894DE01139620E03EE051E2E32FF0E0AB
:101EF00050935700E49120FF03C0E295EF703F5FDD
:101F0000EF708E2F90E0EA3010F0C79601C0C096B7
:101F10008D939D932F5F243149F74FBF8091E80047
:101F2000877F8093E8006AE270E0CE0101960E940C
:101F3000D10B14C0AE014F5F5F4F6091F6010E945C
:101F4000180BBC01009709F440C09091E800977FFE
:101F50009093E80089819A810E94340C8091E80076
:101F60008B778093E80031C0803879F58091E80064
:101F7000877F8093E8008091ED018093F10080914C
:101F8000E8008E778093E8000E94CA0C1EC0811181
:101F90001CC09091F4019230C0F48091E800877FDA
:101FA0008093E8009093ED010E94CA0C8091ED01AE
:101FB000811106C08091E30087FD02C081E001C06D
:101FC00084E08093F1010E94140A8091E80083FF6D
:101FD0000AC08091E800877F8093E8008091EB0041
:101FE00080628093EB00AA960FB6F894DEBF0FBE16
:101FF000CDBFDF91CF911F9108950895CF93809128
:10200000F1018823A1F0C091E900CF709091EC001C
:10201000892F817090FD80E8C82B1092E900809193
:10202000E80083FD0E94AC0ECF70C093E900CF9111
:10203000089590937501809374010895E09174015F
:10204000F0917501309721F00190F081E02D099415
:1020500080E00895E0917401F0917501309721F0CE
:102060000280F381E02D09940895E0917401F091CC
:102070007501309721F00480F581E02D09940895D1
:1020800020917201309173018217930771F0909340
:10209000730180937201E0917401F09175013097A2
:1020A00021F00680F781E02D0994089520917001B8
:1020B000309171018217930771F0909371018093B1
:1020C0007001E0917401F0917501309721F0008466
:1020D000F185E02D0994089508950C946C100E94E8
:1020E000C61B0E943C030C94881C9F92AF92BF9227
:1020F000CF92DF92EF92FF920F931F93CF93DF93D4
:1021000000D000D000D0CDB7DEB70E9454030DE060
:1021100010E0AA24A394B12C902E802F0E94420498
:10212000980129583E4F6901F901F080F826A1F481
:102130000150110988F78FEF89838A831B820E94DF
:10214000CF1B8160782F9D838C8349815A816B815D
:102150008D810E940C112FC09091DA0191FF04C073
:102160008E830E9448048E8125E030E0A501022E76
:1021700001C0440F0A94EAF7E42E4F21C1F02983ED
:102180009A828E2191E009F490E09B830E94CF1BFC
:102190008160782F9D838C8349815A816B818D81E9
:1021A0000E940C11F6018081E826E08204C02150D3
:1021B0003109E0F6BDCF0E946F1F109176010E9499
:1021C0001E101817B9F00E941E10809376012696F3
:1021D0000FB6F894DEBF0FBECDBFDF91CF911F9138
:1021E0000F91FF90EF90DF90CF90BF90AF909F90B6
:1021F0000C94170926960FB6F894DEBF0FBECDBF1C
:10220000DF91CF911F910F91FF90EF90DF90CF90D2
:10221000BF90AF909F900895CF93DF93CDB7DEB777
:102220002B970FB6F894DEBF0FBECDBF4F835887F4
:1022300069877A878B87DE01119686E0FD0111920E
:102240008A95E9F785E0FE01379601900D928A950F
:10225000E1F749815A816B817C818D819E810E9449
:1022600055172B960FB6F894DEBF0FBECDBFDF918A
:10227000CF910895CF93882309F4C2C0C82F823824
:1022800059F40E941E1081FDBBC089E30E942F1AE1
:102290000E94FC1A89E30CC0833879F40E941E1056
:1022A00080FDAEC083E50E942F1A0E94FC1A83E5D0
:1022B0000E94711ACF910C94FC1A843859F40E9430
:1022C0001E1082FD9DC087E40E942F1A0E94FC1AF6
:1022D00087E4EECF8CEF8C0F813A48F48C2F0E946C
:1022E000B22181118DC08C2F0E942F1AE3CF80E282
:1022F0008C0F883048F4C77081E001C0880FCA9500
:10230000EAF70E94B51AD6CF8BE58C0F833078F4AC
:10231000C53A29F0C63A31F083E890E005C081E87B
:1023200090E002C082E890E0CF910C94401088E5E4
:102330008C0F833108F064C0C83A39F1C93A41F1D1
:10234000CA3A49F1CB3A51F1CC3A59F1CD3A61F15F
:10235000C03B69F1CE3A71F1CF3A79F1C13B81F1DD
:10236000C23B89F1C33B91F1C43B99F1C53BA1F15B
:10237000C63BA9F1C73BB1F1C83BB9F1C93BC1F1BB
:10238000CA3BC9F180E090E038C082EE90E035C0F1
:1023900089EE90E032C08AEE90E02FC085EB90E0AD
:1023A0002CC086EB90E029C087EB90E026C08CEC37
:1023B00090E023C08DEC90E020C083E891E01DC048
:1023C0008AE891E01AC082E991E017C084E991E0BF
:1023D00014C081E292E011C083E292E00EC084E278
:1023E00092E00BC085E292E008C086E292E005C070
:1023F00087E292E002C08AE292E0CF910C945610FC
:10240000CF910895882309F44BC0823859F40E9473
:102410001E1081FF45C089E30E942F1A0E94FC1AFA
:1024200089E30CC0833871F40E941E1080FF38C00D
:1024300083E50E942F1A0E94FC1A83E50E94711AFC
:102440000C94FC1A843859F40E941E1082FF28C094
:1024500087E40E942F1A0E94FC1A87E4EFCF9CEFBA
:10246000980F913A58F390E2980F983050F4877093
:1024700091E001C0990F8A95EAF7892F0E94BB1A53
:10248000DFCF9BE5980F933020F480E090E00C9430
:102490004010885A833120F480E090E00C9456106C
:1024A0000895882321F00E94B51A0C94FC1A08950F
:1024B000882321F00E94BB1A0C94FC1A08957F9285
:1024C0008F929F92AF92BF92CF92DF92EF92FF9244
:1024D0000F931F93CF93DF931F92CDB7DEB77C018D
:1024E000C62E772EFC01058102950F701281111105
:1024F0000E94D21A0E94281A882379F0112369F0C9
:1025000080E28C0D883048F082E00E94111A0E940F
:10251000281A91E0D82ED92601C0D12CE72DE295BA
:10252000EF70F0E0E05AFF4F0C94E723872D807F97
:10253000072D0F70882311F00295007F112389F079
:10254000002309F490C180E28C0D883020F4802FA4
:102550000E94B51A03C0802F0E94C51A0E94FC1A5F
:1025600082C18C2D0E940212002309F495C180E2E1
:102570008C0D883020F4802F0E94BB1A03C0802F5E
:102580000E94CB1A0E94FC1A87C1972D907F872D3D
:102590008F70903211F08295807FCC2021F0F1E095
:1025A000CF16B1F01EC0112349F0002309F414C165
:1025B000013009F011C10E94E51A6EC1002319F023
:1025C000013009F469C189830E94E81A89810AC12E
:1025D000112321F0023008F05FC1FEC001115CC17F
:1025E00001C1112321F0002309F4F6C03CC10023EE
:1025F00009F4F8C03EC1872D86958695837090E0DA
:10260000009719F0019761F047C1112321F08C2D3B
:10261000972D937002C080E090E00E9440103CC172
:10262000112321F08C2D972D937002C080E090E053
:102630000E94561031C18C2D112319F00E94771E73
:1026400002C00E94DF1E0E94641F26C1872D837076
:1026500009F052C0111120C18C2D8295869587708A
:10266000880F880F9C2D9F70892E912CA12CB12C46
:10267000082E04C0880C991CAA1CBB1C0A94D2F713
:10268000C4FE14C00FE010E020E030E0B901A80162
:1026900004C0440F551F661F771F8A95D2F7CB01E0
:1026A000BA01609570958095909503C060E070E0E8
:1026B000CB01272D26952695237030E02230310559
:1026C00069F02330310589F0682979298A299B2905
:1026D0002130310571F00E949D18DEC068297929EA
:1026E0008A299B290E94B918D7C00E949D18C5014C
:1026F000B4010E948118D0C0112319F0872D817078
:1027000001C08695882309F4C7C08C2D82958695D3
:102710008770880F880F9C2D9F70892E912CA12C7B
:10272000B12C082E04C0880C991CAA1CBB1C0A944E
:10273000D2F7C4FE14C00FE010E020E030E0B90191
:10274000A80104C0440F551F661F771F8A95D2F752
:10275000CB01BA01609570958095909503C060E0BB
:1027600070E0CB01272D269526952370422F50E04F
:102770004230510569F04330510589F068297929C3
:102780008A299B294130510571F00E94771984C034
:10279000682979298A299B290E9493197DC00E9462
:1027A0007719C501B4010E945B1976C08C2D90E0A9
:1027B000FC01E05EF109E531F10508F050C0E05997
:1027C000FF4F0C94E7230C2D0F70872D8F71112371
:1027D00031F00E94F418802F0E9451125DC00E94B7
:1027E0001519802F0E94581257C0112339F001117A
:1027F00053C0872D8F710E943A194EC0023008F0E5
:102800004BC0F7CF112339F0872D8F710E94F41838
:1028100043C01123C9F3872D8F710E9415193CC045
:10282000112329F0872D8F710E94DF1835C00E9477
:10283000D51832C0112351F0172D1F71812F0E941E
:10284000F41863E0812F0E94081A26C081E00E94DC
:10285000111A023008F182E00E94111A1DC01123E2
:1028600031F0002389F28C2D0E943A1115C000230B
:1028700091F28C2D0E9402120FC0472D4F706C2DCB
:10288000C7010E941E050E94F91706C0472D4F7010
:102890006C2DC7010E942606DD20F9F00E94041A63
:1028A00080FD1BC0F70112820E94FE190E94F418DD
:1028B000C7010E947C140E94FE190F90DF91CF91F6
:1028C0001F910F91FF90EF90DF90CF90BF90AF904E
:1028D0009F908F907F900C9415190F90DF91CF915E
:1028E0001F910F91FF90EF90DF90CF90BF90AF902E
:1028F0009F908F907F9008950F931F93CF93DF93B6
:10290000EC01888199812B813C81232BB9F09F3F79
:1029100011F48F3F99F0CE010E947E05882371F05B
:10292000688179818A810E94FA198C010E94AF190D
:102930000E947618B801CE010E945F12DF91CF91FC
:102940001F910F9108950E94D21A0E94E21A0E94CC
:10295000A71A0E94FC1A0E9415200E94641F80E0A2
:1029600090E00E94401080E090E00C9456100E948D
:10297000C21A0C94A3140E94EF19292F22952F70CC
:1029800030E02C3031054CF42A3031056CF4225003
:10299000310922303105A8F407C02C30310569F027
:1029A0002F30310551F00DC0803F69F018F4803EA2
:1029B00040F409C0843F29F406C093FB882780F9BE
:1029C000089580E0089581E00895CF93DF9300D0CB
:1029D00000D01F92CDB7DEB70F900F900F900F90E1
:1029E0000F90DF91CF910895CF93DF9300D000D067
:1029F00000D0CDB7DEB726960FB6F894DEBF0FBE77
:102A0000CDBFDF91CF9108951F93CF93DF93C091F6
:102A1000850116E080918601C81799F0D0E01C9FCF
:102A2000F0011D9FF00D1124E957FE4F40815181A7
:102A300062817381848195810E94F4142196C7700C
:102A4000E9CFDF91CF911F9108954091B701509147
:102A5000B8016091B9017091BA018091BB01909168
:102A6000BC010C94F4148091BC0182958F7009F024
:102A700054C08091B901882309F44FC08091850129
:102A8000A09186016091B7017091B8014091BA019F
:102A90005091BB01B6E08A1709F43FC090E04115A0
:102AA0005105C1F17F3F11F46F3FA1F1B89FF001D3
:102AB000B99FF00D1124E957FE4F218172132AC0EE
:102AC0002081621327C02281211124C023813481F7
:102AD0002417350710F421503109241B350B283CED
:102AE0003105C0F42091BC012F7020612093BC01FE
:102AF00026E0289FF001299FF00D1124E457FE4F96
:102B000080818F708061808387EB91E00E947C14CC
:102B10000C94041501968770BECF0895CF92DF9272
:102B2000EF92FF920F931F93CF93DF93CDB7DEB752
:102B300062970FB6F894DEBF0FBECDBF8C0185E063
:102B4000F801DE011D9601900D928A95E1F7D801FA
:102B50004C9111965C91119712966C911297139665
:102B6000CD90DC9014973091B7017091B8018091AD
:102B7000BA019091BB01009709F46BC17F3F19F432
:102B80003F3F09F466C1E090B901EE2009F4C0C0EE
:102B90002091BC01C816D90628F0F601E81BF90BF4
:102BA000CF0104C0809590958C0D9D1DFF24F3945A
:102BB000883C910578F0F12C207F09F0C6C07C2D6F
:102BC000D98AC88A89890E94E51487EB91E00E941E
:102BD0007C14B1C0822F807F09F046C0751314C0E9
:102BE000341312C0611110C02F7020612093BC01FA
:102BF0000E94251587EB91E00E947C148091BC0116
:102C0000D80115968C932EC0CD2819F15F3F11F491
:102C10004F3FF9F0F62E61111CC080918501209183
:102C2000860136E0821709F45AC090E0389FF0011F
:102C3000399FF00D1124E957FE4F7181571306C0DB
:102C40007081471303C07281711103C001968770B0
:102C5000E9CFF62E662309F418C18091BC0181608A
:102C60008093BC01F12C11C1751308C0341306C048
:102C7000611104C08091BC01D801C3C04D875E873B
:102C80008D859E856A8B0E94BB146A898823E1F139
:102C90006623D1F12091BC01822F82958F7090E044
:102CA000029774F08091B7019091B80198878F8353
:102CB0001986DB86CA862C87CE0107960E947C1473
:102CC00086E0F801A7EBB1E001900D928A95E1F75B
:102CD0000E9433150E942515FF24F394D6C04D871A
:102CE0005E878D859E850E94EF19292F22952F7072
:102CF00030E0223031050CF0BCC09F7009F0B6C046
:102D0000805E883008F4C1C0C8010E947C14E4CF02
:102D1000C816D90608F453C0F601E81BF90BCF0119
:102D2000883C910508F450C0F12C7C2DD98AC88AC2
:102D300089890E94E514E7EBF1E086E0DF011D924E
:102D40008A95E9F70E942515A0C0751314C03413A5
:102D500012C0611110C08091BC01F8018583C801C7
:102D60000E947C1486E0E7EBF1E0DF011D928A957A
:102D7000E9F7FE2C8AC04D875E878D859E856A8B1C
:102D80000E94BB146A89882309F4BECF662309F424
:102D9000BBCF2091BC01822F82958F7090E002976B
:102DA0000CF48ECF8091B7019091B8019A838983FA
:102DB0001B82DD82CC822E83CE0101967FCF80954F
:102DC00090958C0D9D1DACCFF62E662309F49CCFFB
:102DD00075132EC034132CC02091BC0120FD1FC0E0
:102DE000822F82958F70D9F0D80115962C93159764
:102DF0008F3049F08F5F982F9295907F822F8F7040
:102E0000892B15968C93C8010E947C1486E0F801EA
:102E1000A7EBB1E001900D928A95E1F793CF86E0A0
:102E2000F801A7EBB1E001900D928A95E1F72DC072
:102E30004D875E878D859E850E94BB14811140CF92
:102E40008091BC0181608093BC01C8010E947C1408
:102E50001CC0662309F458CF4D875E878D859E85FB
:102E60000E94BB14882309F44FCF2ACF811148CF89
:102E70000CC0243031050CF047CF9F7009F440CFCF
:102E8000F8019581907F09F03BCF8F2D62960FB6A8
:102E9000F894DEBF0FBECDBFDF91CF911F910F9190
:102EA000FF90EF90DF90CF9008951F93CF93DF9323
:102EB000CDB7DEB72C970FB6F894DEBF0FBECDBFEF
:102EC0004F83588769877A878B879C87CE010796BF
:102ED0000E948E15882369F08F8198852A853B850D
:102EE000232BF1F19F3F09F063C08F3F09F060C0D1
:102EF00037C086E0FE013796DE01119601900D92F3
:102F00008A95E1F76F817885EA85FB85309741F1F5
:102F10007F3F11F46F3F21F12091860130E0C9011C
:102F20000196877099274091850150E08417950795
:102F300009F447C069837A83FD83EC8396E0929F0E
:102F4000D001939FB00D1124A957BE4FFE013196B9
:102F500001900D929A95E1F7809386010E940415E5
:102F600016E080918501909186018917C1F1189F23
:102F7000C001112489579E4F0E948E15882379F134
:102F8000E09185011E9FF0011124E957FE4F408119
:102F9000518162817381848195810E94F4148091B2
:102FA000850190E001968770992780938501D9CF9C
:102FB0004F81588569857A858B859C850E94F4149C
:102FC000CFCF0E94B7141092860110928501E7EBD3
:102FD000F1E086E0DF011D928A95E9F7C1CF2C96DA
:102FE0000FB6F894DEBF0FBECDBFDF91CF911F911A
:102FF0000895EF92FF920F931F93CF93DF938C016D
:10300000009709F46CC0F12CEE24E394E8012196BA
:10301000F8018491843740F4843008F051C0813045
:1030200081F0823019F15BC0853709F444C0A8F102
:103030009CE7980F903708F052C08F770E940212D9
:1030400041C00E5F1F4FFE01C49180E28C0F88309B
:1030500048F4C7708E2D01C0880FCA95EAF70E9408
:10306000D51A14C08C2F0E943A112DC00E5F1F4F2D
:10307000FE01C49180E28C0F883058F4C7708E2D09
:1030800001C0880FCA95EAF70E94DB1A0E94FC1A59
:103090001AC08C2F0E94021216C00E5F1F4FFE0135
:1030A000C491CC2381F08FE99FE00197F1F700C034
:1030B0000000C150F6CF0E5F1F4FFE01F49003C019
:1030C0000E943A118E018F2D882309F49FCFEFE9DA
:1030D000FFE03197F1F700C000008150F5CFDF919C
:1030E000CF911F910F91FF90EF90089508956093F5
:1030F000C1017093C2018093C3019093C4010C94E9
:10310000A3140F931F930091C1011091C20120914C
:10311000C3013091C401DC01CB01802B912BA22B88
:10312000B32B8093C1019093C201A093C301B093CC
:10313000C4011F910F910C94A3140F931F9300913E
:10314000C1011091C2012091C3013091C401DC0181
:10315000CB0180239123A223B3238093C1019093B9
:10316000C201A093C301B093C4011F910F910C94AD
:10317000A3140F931F930091C1011091C2012091DC
:10318000C3013091C401DC01CB0180279127A22724
:10319000B3278093C1019093C201A093C301B09360
:1031A000C4011F910F910C94A3141092BD011092B1
:1031B000BE011092BF011092C0010C94A31441E013
:1031C00050E060E070E004C0440F551F661F771F99
:1031D0008A95D2F74093BD015093BE016093BF0121
:1031E0007093C0010C94A31441E050E060E070E0E3
:1031F00004C0440F551F661F771F8A95D2F7809130
:10320000BD019091BE01A091BF01B091C001482BBA
:10321000592B6A2B7B2B4093BD015093BE016093C9
:10322000BF017093C0010C94A31441E050E060E032
:1032300070E004C0440F551F661F771F8A95D2F7B0
:1032400040955095609570958091BD019091BE011B
:10325000A091BF01B091C001482359236A237B2369
:103260004093BD015093BE016093BF017093C001B4
:103270000C94A31441E050E060E070E004C0440FFF
:10328000551F661F771F8A95D2F78091BD019091D7
:10329000BE01A091BF01B091C001482759276A27FC
:1032A0007B274093BD015093BE016093BF01709393
:1032B000C0010C94A3140F931F930091BD011091B2
:1032C000BE012091BF013091C001DC01CB01802BF8
:1032D000912BA22BB32B8093BD019093BE01A093A1
:1032E000BF01B093C0011F910F910C94A3140F93D1
:1032F0001F930091BD011091BE012091BF0130913B
:10330000C001DC01CB0180239123A223B32380934E
:10331000BD019093BE01A093BF01B093C0011F9166
:103320000F910C94A3140F931F930091BD01109162
:10333000BE012091BF013091C001DC01CB0180278B
:103340009127A227B3278093BD019093BE01A0933C
:10335000BF01B093C0011F910F910C94A314089565
:10336000CF92DF92EF92FF920F931F93CF93DF9351
:103370008C01C090C101D090C201E090C301F090D7
:10338000C4018091BD019091BE01A091BF01B09197
:10339000C001C82AD92AEA2AFB2ACFE1D0E0D70106
:1033A000C6010C2E04C0B695A795979587950A94EB
:1033B000D2F780FF06C0B8018C2F0E947C080197CD
:1033C00021F4219760F780E001C08C2FDF91CF912D
:1033D0001F910F91FF90EF90DF90CF900895CF93C2
:1033E000DF93EC010E94B019BE010E947C08DF91BE
:1033F000CF910895CB010E94EF1908958091C501E6
:1034000085958595859508958091C5018770089566
:1034100098E0899F90011124262B2093C5010C94DC
:10342000F4182091C501809582238093C501982FBF
:10343000977069F430E0482F552747FD50952417C1
:10344000350729F08595859585950C94151908956E
:103450009091C501977081E009F480E00895909102
:103460000C01992321F090910D01911109C0209137
:103470000E0130910F01F90132969FEF40E01FC01D
:10348000982F9695969596959F3050F5E0910E0160
:10349000F0910F01E90FF11D877021E030E0A901E3
:1034A00002C0440F551F8A95E2F7CA019181892B0A
:1034B000818308959F3F39F04F5F4E3041F0519125
:1034C0005813F8CF0DC05111F7CF942FF5CF9F3F70
:1034D00039F0F901E90FF11D97FDFA9582830895FE
:1034E000089590910C01992321F090910D01911173
:1034F00009C020910E0130910F01F9013296205F31
:103500003F4F1FC0982F9695969596959F30F0F453
:10351000E0910E01F0910F01E90FF11D877021E09C
:1035200030E0A90102C0440F551F8A95E2F7CA0195
:10353000809591818923818308953196E217F3075D
:1035400029F090819813F9CF1082F7CF089581E088
:1035500090E0E0910E01F0910F01E80FF91F108249
:10356000019680319105A9F708959091D901892B91
:103570008093D901089580959091D90189238093F2
:10358000D90108951092D90108959091D801892BFD
:103590008093D801089580959091D80189238093D4
:1035A000D80108951092D80108959091D701892BE0
:1035B0008093D701089580959091D70189238093B6
:1035C000D70108951092D70108958093C6010895F8
:1035D0001092C601089580910E0190910F01FC0197
:1035E00031969C01205F3F4F80E0919191118F5F58
:1035F000E217F307D1F70895E0910E01F0910F0162
:103600008091D9018083E0910E01F0910F019081AA
:103610008091D801892B8083E0910E01F0910F01F8
:1036200090818091D701892B80838091C601882366
:1036300061F0E0910E01F0910F019081892B808360
:103640000E94EB1A81111092C60180910E01909197
:103650000F010C942A1020E0009739F0AC01415082
:103660005109842395232F5FF7CF822F0895CF929E
:10367000DF92EF92FF926C01EE24FF24C114D1047B
:10368000E104F10421F0C701B60120E101C020E00E
:10369000C72ED82EE92EFF24C114D104E104F10471
:1036A00019F0285FC701B6016B017C0154E0F69464
:1036B000E794D794C7945A95D1F7C114D104E10483
:1036C000F10419F02C5FC701B6016B017C0142E0E7
:1036D000F694E794D794C7944A95D1F7C114D104CE
:1036E000E104F10419F02E5FC701B601DC01CB0142
:1036F000B695A79597958795892B8A2B8B2B09F0E3
:103700002F5F822FFF90EF90DF90CF9008958091F0
:10371000F101843021F11092DB0120E488E190E096
:103720000FB6F894A895809360000FBE20936000B8
:1037300080E00E94170983B7817F846083BF83B7CD
:10374000816083BF7894889583B78E7F83BF88E13B
:103750000FB6F89480936000109260000FBE089539
:10376000089508950E94B01B0E9454030E94B11B4B
:103770000E94490491E0811101C090E0892F0895D1
:103780000E94B7140E941E100C94170982E084BD99
:1037900093E095BD9AEF97BD80936E0008952FB783
:1037A000F8948091DC019091DD01A091DE01B0914F
:1037B000DF012FBF0895CF92DF92EF92FF920F9318
:1037C0001F932FB7F8944091DC015091DD01609177
:1037D000DE017091DF012FBF6A017B01EE24FF241F
:1037E0008C0120E030E0C016D106E206F30610F4AA
:1037F000415051099A01281B390BC9011F910F91A2
:10380000FF90EF90DF90CF9008951F920F920FB628
:103810000F9211248F939F93AF93BF938091DC01FC
:103820009091DD01A091DE01B091DF010196A11D13
:10383000B11D8093DC019093DD01A093DE01B09374
:10384000DF01BF91AF919F918F910F900FBE0F90AD
:103850001F9018950E941B0DF8942FEF87EA91E6B0
:10386000215080409040E1F700C0000087E090EBDD
:10387000DC018093FB019093FC01A093FD01B093C8
:10388000FE019CE088E10FB6F894A8958093600053
:103890000FBE90936000FFCFEF92FF920F931F93A4
:1038A000CF93DF93D82FCDE08C2F0E94420405E008
:1038B00010E0E82EF12CC701002E02C095958795E7
:1038C0000A94E2F780FF09C0602F7C2F80E00E94FD
:1038D0002706D81302C081E006C00150110958F72D
:1038E000C15010F780E0DF91CF911F910F91FF90B1
:1038F000EF900895CF93C82F8CE20E944C1C882330
:1039000021F08C2FCF910C944C1C80E0CF91089526
:10391000CF930E94CF1D811102C00E94B51DC5E644
:10392000C15049F00E9454038FE39CE90197F1F7DD
:1039300000C00000F5CF89E20E947A1C811113C1FA
:103940008AE20E947A1C81110E94B51D85E00E94C6
:103950007A1C81110E942A1C0E94DA1D8093DA01D0
:1039600087E00E947A1C8823A9F18BE10E947A1CCF
:10397000882351F08091DA0181FB222720F991E020
:10398000922790FB81F90EC08EE00E947A1C88235A
:1039900061F08091DA0182FB222720F991E09227E1
:1039A00090FB82F98093DA0115C080E10E947A1CB5
:1039B0009091DA01882341F093FB222720F981E0DE
:1039C000822780FB93F904C0892F809580FB90F9B2
:1039D0009093DA018091DA010E94DE1D0E94EC1DB5
:1039E0008093FA0180EE0E947A1C882341F0809136
:1039F000FA01982F909590FB80F98093FA0189E362
:103A00000E947A1C882359F08091FA0181FB2227B9
:103A100020F991E0922790FB81F98093FA0182EEE0
:103A20000E947A1C882359F08091FA0182FB222798
:103A300020F991E0922790FB82F98093FA0186EEBB
:103A40000E947A1C882359F08091FA0183FB222777
:103A500020F991E0922790FB83F98093FA0183EE9D
:103A60000E947A1C882359F08091FA0184FB222756
:103A700020F991E0922790FB84F98093FA0185E385
:103A80000E947A1C882359F08091FA0185FB222735
:103A900020F991E0922790FB85F98093FA0181E368
:103AA0000E947A1C882359F08091FA0186FB222714
:103AB00020F991E0922790FB86F98093FA0181E149
:103AC0000E947A1C882359F08091FA0187FB2227F3
:103AD00020F991E0922790FB87F98093FA01809179
:103AE000FA010E94F01D8091FA0187FB882780F976
:103AF00080930D0187E20E947A1CC82F8EE10E94FC
:103B00007A1C8111C2608FE10E947A1C8111C4600D
:103B100080E20E947A1C8111C86081E20E947A1CB6
:103B20008111C06182E20E947A1C8111C06283E22D
:103B30000E947A1C8111C06484E20E947A1C88234E
:103B400011F0C06802C0CC2329F08C2F0E94E71D21
:103B50006C2F03C00E94E31D682F70E080E090E0AE
:103B6000CF910C947718CF9108956DEE7EEF80E0A1
:103B700090E00E94212460E082E090E00E940F2407
:103B800060E083E090E00E940F2460E084E090E039
:103B90000E940F2460E085E090E00C940F2480E008
:103BA00090E00E94092421E08D3E9E4F09F020E024
:103BB000822F089582E090E00C940124682F82E027
:103BC00090E00C940F2483E090E00C940124682F83
:103BD00083E090E00C940F2484E090E00C940124A6
:103BE000682F84E090E00C940F248091E20180FF24
:103BF0000BC06091130185E0689FB0011124759599
:103C00006795759567952BC081FF09C06091130179
:103C100085E0689FB00111247595679520C082FFEB
:103C200007C06091130185E0689FB001112417C09F
:103C30009091E3019923D1F060911201961788F7D2
:103C40002091130185E0289F90011124929FA001EB
:103C5000939F500D112470E0CA010E94D323603855
:103C6000710540F46115710539F002C065E070E03E
:103C7000862F08958FE7089581E008958091E201ED
:103C800080FF08C06091110170E07595679575958A
:103C9000679521C081FF06C06091110170E07595A4
:103CA000679519C082FF04C06091110170E010C0D7
:103CB0009091E3019923C1F0609110019617A0F74C
:103CC00080911101899FC001112470E00E94D323CB
:103CD0006038710528F46115710521F0862F08956B
:103CE0008FE7089581E0089561E070E0F4CF803FB0
:103CF00021F40E94F51D819504C0813F29F40E94A2
:103D0000F51D8093E6010895823F21F40E94F51D80
:103D1000819504C0833F29F40E94F51D8093E5013D
:103D20000895893F19F40E943E1E05C08A3F31F470
:103D30000E943E1E81958093E70108958B3F21F4F8
:103D40000E943E1E819504C08C3F29F40E943E1EB5
:103D50008093E8010895843F21F48091E40181601B
:103D600017C0853F21F48091E401826011C0863F35
:103D700021F48091E40184600BC0873F21F480919D
:103D8000E401886005C0883F31F48091E4018061DE
:103D90008093E40108958D3F21F48091E2018160D8
:103DA0000BC08E3F21F48091E201826005C08F3FFD
:103DB00029F48091E20184608093E2010895803FBC
:103DC00039F48091E60187FF6CC01092E60169C06A
:103DD000813F29F48091E6011816BCF362C09091EE
:103DE000E501823F29F497FF5CC01092E50159C0BC
:103DF000833F19F41916CCF354C0893F41F48091E4
:103E0000E70118160CF04DC01092E7014AC08A3F36
:103E100029F48091E70187FF44C0F6CF8B3F39F446
:103E20008091E80187FF3DC01092E8013AC08C3FC5
:103E300029F48091E8011816BCF333C0843F21F4C3
:103E40008091E4018E7F17C0853F21F48091E401C9
:103E50008D7F11C0863F21F48091E4018B7F0BC0E0
:103E6000873F21F48091E401877F05C0883F31F4CA
:103E70008091E4018F7E8093E40113C08D3F21F493
:103E80008091E2018E7F0BC08E3F21F48091E20190
:103E90008D7F05C08F3F29F48091E2018B7F809355
:103EA000E2018091E50181110EC08091E60181114E
:103EB0000AC08091E701811106C08091E80181115B
:103EC00002C01092E301089584EE91E00E94351043
:103ED0000E94CF1B9093E1018093E00108951F930E
:103EE000CF93DF938091E0019091E1010E94DB1B71
:103EF000AC019091E301992321F02091140130E06D
:103F000006C0209115018AE0289F900111244217D4
:103F1000530708F486C08091E501C091E601D09175
:103F2000E7011091E801811107C0C11176C0D111DC
:103F300074C0111172C075C09F3F19F09F5F9093BC
:103F4000E301181624F40E94F51D8093E501809189
:103F5000E50187FF05C00E94F51D81958093E5016D
:103F60001C1624F40E94F51D8093E6018091E60161
:103F700087FF05C00E94F51D81958093E601609141
:103F8000E501662339F1C091E601CC2319F17727C9
:103F900067FD7095872F972F0E94E42223E333E378
:103FA00043E35FE30E9448230E94B1226093E5014E
:103FB0006C2F772767FD7095872F972F0E94E4223B
:103FC00023E333E343E35FE30E9448230E94B122EB
:103FD0006093E6011D1624F40E943E1E8093E701C3
:103FE0008091E70187FF05C00E943E1E8195809366
:103FF000E701111624F40E943E1E8093E80180918F
:10400000E80187FF05C00E943E1E81958093E8016C
:10401000DF91CF911F910C94641F9F3F09F08ECFC9
:1040200096CFDF91CF911F910895E4EEF1E085E006
:10403000DF011D928A95E9F71092E3011092E201E7
:104040000895833081F128F4813059F08230D1F025
:104050000895853009F449C0B8F1863009F456C096
:10406000089580911501262F30E0280F311D2F3F34
:10407000310524F4680F6093150108958FEF809344
:104080001501089580911401262F30E0280F311D6D
:104090002F3F310524F4680F6093140108958FEFCA
:1040A00080931401089580911301262F30E0280F8A
:1040B000311D2F3F310524F4680F609313010895DB
:1040C0008FEF80931301089580911201262F30E025
:1040D000280F311D2F3F310524F4680F6093120122
:1040E00008958FEF80931201089580911101262F7A
:1040F00030E0280F311D2F3F310524F4680F609305
:10410000110108958FEF809311010895809110019E
:10411000262F30E0280F311D2F3F310524F4680F82
:104120006093100108958FEF8093100108958330FC
:1041300011F128F4813049F0823091F008958530F2
:1041400081F120F18630C1F1089580911501681741
:1041500020F4861B8093150108951092150108958F
:1041600080911401681720F4861B80931401089530
:1041700010921401089580911301681720F4861B92
:1041800080931301089510921301089580911201F4
:10419000681720F4861B8093120108951092120173
:1041A000089580911101681720F4861B80931101F6
:1041B000089510921101089580911001681720F45C
:1041C000861B8093100108951092100108950F939B
:1041D0001F938D3109F46BC008F03FC08E3009F495
:1041E0007FC0C0F4873009F469C068F4863009F0F4
:1041F000B1C08091DA01817F8E7F8093DA0181E006
:104200008093EA01A8C0883009F4A2C08B3009F479
:104210009FC0A0C0863109F49BC078F4803109F4B6
:1042200072C0813109F096C00E94B71490910D01BF
:1042300081E0892780930D018BC0893109F488C002
:104240008B3109F087C08091DA0181FB222720F9A8
:1042500091E0922790FB81F94CC0853309F470C03E
:1042600048F4873209F46CC008F459C0893209F463
:1042700067C070C0833438F48A3308F04EC0883386
:1042800009F466C067C0833409F45AC0883409F061
:1042900061C00E94B7140FEF13ED20E301501040EE
:1042A0002040E1F700C000000E942A1C51C00E947B
:1042B0006B220E941E100E9417094AC09091DA01D9
:1042C000892F8095817080FB90F929F09660986025
:1042D0009093DA0140C0997F977F9093DA0138C0BC
:1042E0008091DA0182FB222720F991E0922790FB4E
:1042F00082F98093DA01992359F18091DA01816082
:104300008093DA0125C08091DA0183FB222720F90E
:1043100091E0922790FB83F9ECCF895301C08D5136
:1043200041E050E060E070E08A019B0104C0000FB2
:10433000111F221F331F8A95D2F7C901B80104C08B
:1043400061E070E080E090E00E9477180E94B7146E
:1043500081E001C080E01F910F91089580E00895F1
:1043600080E00895CF93C82F8091EA01813079F0E1
:1043700018F08230E9F187C0E0910E01F0910F0151
:104380008081813169F0823209F07FC009C0E091FB
:104390000E01F0910F018081813111F0823261F4C0
:1043A0008C2F0E94AE21811104C08C2F0E94E72027
:1043B0001DC081E090E01AC08C2F0E94B0218111B5
:1043C00014C0C43179F048F4CB3079F0C03109F031
:1043D00060C082E08093EA0108C0C93219F0C83396
:1043E00021F057C01092EA0154C081E0817053C09F
:1043F000C93289F118F5C43171F1A8F4C73009F058
:1044000046C08AE08093150194E19093140193E0F3
:10441000909313018093120188E08093110188E248
:104420008093100134C0CE51C63088F5EC2FF0E0F7
:10443000E65DFE4F80818093E90129C0CE34E9F02A
:1044400020F4CB3421F56AE013C0C13579F0C235D0
:10445000F1F461E00DC08091E901882319F0109218
:10446000E90115C081E08093EA0115C061E006C052
:104470008091E9010E9421200AC06AE08091E9014F
:104480000E94972004C01092EA0180E004C081E0FD
:1044900002C080E0ABCFCF910895E1E8F0E08081E9
:1044A000886080838081816080838FB7F89493E0F7
:1044B0009093890090ED909388008FBF0895EFE668
:1044C000F0E08081826080830895EFE6F0E08081F3
:1044D0008D7F80830895EFE6F0E0908182E0892768
:1044E000808308951F920F920FB60F9211242F937D
:1044F0003F934F935F936F937F938F939F93AF936C
:10450000BF93EF93FF938091EB019091EC010196A3
:104510009093EC018093EB01811103C082E00E9433
:104520001709E091EC01E695E695F0E0EA53FB4FC0
:10453000E4918091EB018E1303C080E00E94170983
:10454000FF91EF91BF91AF919F918F917F916F916B
:104550005F914F913F912F910F900FBE0F901F9041
:10456000189504D06894B1118DC0089570D088F06A
:104570009F5790F0B92F9927B751A0F0D1F0660F4F
:10458000771F881F991F1AF0BA95C9F712C0B1306A
:1045900081F077D0B1E0089574C0672F782F882715
:1045A000B85F39F0B93FCCF3869577956795B395A9
:1045B000D9F73EF490958095709561957F4F8F4F18
:1045C0009F4F0895E89409C097FB3EF4909580951D
:1045D000709561957F4F8F4F9F4F9923A9F0F92FC9
:1045E00096E9BB279395F695879577956795B79547
:1045F000F111F8CFFAF4BB0F11F460FF1BC06F5F2D
:104600007F4F8F4F9F4F16C0882311F096E911C03E
:10461000772321F09EE8872F762F05C0662371F05F
:1046200096E8862F70E060E02AF09A95660F771F73
:10463000881FDAF7880F9695879597F9089557FDA3
:104640009058440F551F59F05F3F71F04795880F00
:1046500097FB991F61F09F3F79F087950895121697
:1046600013061406551FF2CF4695F1DF08C0161643
:1046700017061806991FF1CF8695710561050894F4
:104680000895E894BB2766277727CB0197F908950B
:104690000BD078C069D028F06ED018F0952309F0BF
:1046A0005AC05FC01124EECFCADFA0F3959FD1F3AB
:1046B000950F50E0551F629FF001729FBB27F00DD0
:1046C000B11D639FAA27F00DB11DAA1F649F662725
:1046D000B00DA11D661F829F2227B00DA11D621F74
:1046E000739FB00DA11D621F839FA00D611D221F2E
:1046F000749F3327A00D611D231F849F600D211D12
:10470000822F762F6A2F11249F5750408AF0E1F0B4
:1047100088234AF0EE0FFF1FBB1F661F771F881FFD
:1047200091505040A9F79E3F510570F014C0AACF98
:104730005F3FECF3983EDCF3869577956795B795E8
:10474000F795E7959F5FC1F7FE2B880F911D969512
:10475000879597F9089597F99F6780E870E060E082
:1047600008959FEF80EC089500240A94161617060A
:1047700018060906089500240A9412161306140652
:1047800005060895092E0394000C11F4882352F0B5
:10479000BB0F40F4BF2B11F460FF04C06F5F7F4F6D
:1047A0008F4F9F4F089597FB072E16F4009407D064
:1047B00077FD09D00E94ED2307FC05D03EF49095CB
:1047C00081959F4F0895709561957F4F0895EE0FE5
:1047D000FF1F0590F491E02D0994AA1BBB1B51E12A
:1047E00007C0AA1FBB1FA617B70710F0A61BB70B61
:1047F000881F991F5A95A9F780959095BC01CD0106
:104800000895F999FECF92BD81BDF89A992780B598
:104810000895A8E1B0E042E050E00C942924262F4E
:10482000F999FECF92BD81BDF89A019700B40216A6
:1048300039F01FBA20BD0FB6F894FA9AF99A0FBE54
:1048400008950196272F0E9410240C940F24DC0158
:10485000CB01FC01F999FECF06C0F2BDE1BDF89A8B
:10486000319600B40D9241505040B8F70895F89435
:02487000FFCF78
:1048720002201909A709840950091C090101C7016D
:1048820028080A03140A3F4D363987043A040404FF
:10489200CB035E0377039003A90301020304050619
:0448A20007080900FA
:00000001FF
